:086146000020406080A0C0FFB2
:105F3800C204C201C200C205C20FE4F555C208C2BC
:085F480009C203C20DC20C22C4
:10591200856382856283740693F8E675F015A4FFA9
:10592200740193FA7402932FF9EA35F0AF01F5642A
:105932008F658F82F583E5822408F582E43583F54D
:0D59420083E0FFD39404400590048BEFF048
:01594F002235
:1058500090048BEEF0A3EFF0F5828E83A3A3A374E4
:105860000193FA740293F5828A837F0212293B9096
:10587000048BE0FCA3E0F5828C83740693F8E6FFCA
:10588000A3A3A3740193FA740293F5828A83022975
:015890003BDC
:105B8D003007247E5F7F80EFB5630BEEB5620712A1
:105B9D0058507F0A80137E5F7F8C1258507F0A12F7
:105BAD00560F7F090257407F091257407F09125641
:025BBD000F22B5
:10607E00E49010B5F0C203200705D207125B8D0223
:02608E005912A5
:105FC600856382856283740693F8A607AF63AE6223
:065FD6001258500259129E
:105A0600300735856382856283740693F8EF26F640
:105A1600856382856283740693F8E6FFB41804E40E
:105A2600F68006EFB4FF027617856382856283747B
:095A36000693F8E6FF125FC62298
:0A6129007F0B1257407F0B02560F48
:1056F70012613312609075BB06C2EDD2EC30EDFD3E
:10570700E5BFD3947F4004D2108002C21075BB0757
:10571700C2EDD2EC30EDFDE5BFD3947F4004D2114A
:105727008002C2113010093011037F24227F252205
:085737003011037F26227F27B9
:01573F002247
:085E0800AB07AF031BEF601AAA
:105E10009004791228C30000445C90047974FF1246
:0A5E20002884EC4D4E4F60E280F044
:015E2A002255
:100C9A00E4F5841256F790116EEFF012556D125268
:100CAA00F41260A212595012546F12508812619CA9
:100CBA0043E602905F80E493FB740193FA74029313
:100CCA00F9900008122690D394054007900008E492
:100CDA001226F1E4900474F0A3F0E4900476F0A3F1
:100CEA00F0900474E0FEA3E0FF905F8075F00C12B0
:100CFA002905EE75F00CA42583F583E493FB7401B2
:100D0A0093FA740293F9900476E0FCA3E0F5828CDE
:100D1A008374151228F4E92582F9EA3583FA122731
:100D2A00DC54FEFDE5F08DF012283F905F8075F0EF
:100D3A000CEF122905EE75F00CA42583F583E493D4
:100D4A00FB740193FA740293F9900476E0FEA3E02F
:100D5A00F5828E8374151228F4E92582F9EA35831F
:100D6A00FA1227DC54FDFFE5F08FF012283F9004B9
:100D7A0074E0FEA3E0FF905F8075F00C122905EE87
:100D8A0075F00CA42583F583E493FB740193FA743C
:100D9A000293F9900476E0FCA3E0F5828C83741543
:100DAA001228F4E92582F9EA3583FA1227DC54FB82
:100DBA00FDE5F08DF012283F905F8075F00CEF1280
:100DCA002905EE75F00CA42583F583E493FB7401E1
:100DDA0093FA740293F9900476E0FEA3E0F5828E0A
:100DEA008374151228F4E92582F9EA3583FA122761
:100DFA00DC54F7FFE5F08FF012283F900474E0FE10
:100E0A00A3E0FF905F8075F00C122905EE75F00CD7
:100E1A00A42583F583E493FB740193FA740293F98E
:100E2A00900476E0FCA3E0F5828C8374151228F412
:100E3A00E92582F9EA3583FA1227DC54EFFDE5F059
:100E4A008DF012283F905F8075F00CEF122905EEA5
:100E5A0075F00CA42583F583E493FB740193FA746B
:100E6A000293F9900476E0FEA3E0F5828E8374156E
:100E7A001228F4E92582F9EA3583FA1227DC54DFCD
:100E8A00FFE5F08FF012283F900474E0FEA3E0FF24
:100E9A00905F8075F00C122905EE75F00CA425837D
:100EAA00F583E493FB740193FA740293F990047640
:100EBA00E0FCA3E0F5828C8374151228F4E92582FC
:100ECA00F9EA3583FA1227DC54BFFDE5F08DF012FA
:100EDA00283F905F8075F00CEF122905EE75F00C33
:100EEA00A42583F583E493FB740193FA740293F9BE
:100EFA00900476E0FEA3E0F5828E8374151228F43E
:100F0A00E92582F9EA3583FA1227DCFFE5F054FE77
:100F1A00FEEF547FFFEE8FF012283F900474E0FE3C
:100F2A00A3E0FF905F8075F00C122905EE75F00CB6
:100F3A00A42583F583E493FB740193FA740293F96D
:100F4A00900476E0FCA3E0F5828C8374151228F4F1
:100F5A00E92582F9EA3583FA1227DCFDE5F054F92E
:100F6A008DF012283F905F8075F00CEF122905EE84
:100F7A0075F00CA42583F583E493FB740193FA744A
:100F8A000293F9900476E0FEA3E0F5828E8374154D
:100F9A001228F4E92582F9EA3583FA1227DCFFE5FB
:100FAA00F054E78FF012283F900474E0FEA3E0FFAC
:100FBA00905F8075F00C122905EE75F00CA425835C
:100FCA00F583E493FB740193FA740293F99004761F
:100FDA00E0FCA3E0F5828C8374151228F4E92582DB
:100FEA00F9EA3583FA1227DCFDE5F0549F8DF012F9
:100FFA00283F905F8075F00CEF122905EE75F00C12
:10100A00A42583F583E493FB740193FA740293F99C
:10101A00900476E0FEA3E0FF7C007D15122713E919
:10102A002FF9EA3EFAE92402F9E43AFA1227DC54E3
:10103A00F8FDE5F08DF012283F900474E0FCA3E07F
:10104A00905F8075F00C122905EC75F00CA42583CD
:10105A00F583E493FB740193FA7402932FF9EA3E41
:10106A00FAE92402F9E43AFA1227DC54074450FF59
:10107A00E48FF012283F900474E0FEA3E0905F80B2
:10108A0075F00C122905EE75F00CA42583F583E49E
:10109A0093FB740193FA740293F9900476E0FEA329
:1010AA00E0FF7C007D15122713E92FF9EA3EFA903A
:1010BA000004E41226F1900474E0FCA3E0FD905FC2
:1010CA008075F00C122905EC75F00CA42583F583C4
:1010DA00E493FB740193FA7402932FF9EA3EFA90AF
:1010EA000005E41226F1905F8075F00CED122905D7
:1010FA00EC75F00CA42583F583E493FB740193FA51
:10110A00740293F9900476E0FEA3E0FF7C007D155B
:10111A00122713E92FF9EA3EFA900006E41226F1A3
:10112A00900474E0FCA3E0FD905F8075F00C122936
:10113A0005EC75F00CA42583F583E493FB74019305
:10114A00FA7402932FF9EA3EFA900007E41226F1A4
:10115A00905F8075F00CED122905EC75F00CA42552
:10116A0083F583E493FB740193FA740293F9900470
:10117A0076E0FEA3E0FF7C007D15122713E92FF924
:10118A00EA3EFA900008E41226F1900474E0FCA307
:10119A00E0FD905F8075F00C122905EC75F00CA447
:1011AA002583F583E493FB740193FA7402932FF970
:1011BA00EA3EFA900009E41226F1905F8075F00C7D
:1011CA00ED122905EC75F00CA42583F583E493FB55
:1011DA00740193FA740293F9900476E0FEA3E0FF97
:1011EA007C007D15122713E92FF9EA3EFA90000ACE
:1011FA00E41226F1900474E0FCA3E0FD905F807590
:10120A00F00C122905EC75F00CA42583F583E49300
:10121A00FB740193FA7402932FF9EA3EFA90000BD9
:10122A00E41226F1905F8075F00CED122905EC7539
:10123A00F00CA42583F583E493FB740193FA7402FA
:10124A0093F9900476E0FEA3E0FF7C007D15122757
:10125A0013E92FF9EA3EFA90000CE41226F1900401
:10126A0074E0FCA3E0FD905F8075F00C122905EC98
:10127A0075F00CA42583F583E493FB740193FA7447
:10128A0002932FF9EA3EFA90000DE41226F1905FDC
:10129A008075F00CED122905EC75F00CA42583F588
:1012AA0083E493FB740193FA740293F9900476E051
:1012BA00FEA3E0FF7C007D15122713E92FF9EA3E11
:1012CA00FA90000EE41226F1900474E0FCA3E0FD0B
:1012DA00905F8075F00C122905EC75F00CA425833B
:1012EA00F583E493FB740193FA7402932FF9EA3EAF
:1012FA00FA90000FE41226F1905F8075F00CED125F
:10130A002905EC75F00CA42583F583E493FB74019D
:10131A0093FA740293F9900476E0FEA3E0FF7C004E
:10132A007D15122713E92FF9EA3EFA900010E4120C
:10133A0026F1900474E0FCA3E0FD905F8075F00C48
:10134A00122905EC75F00CA42583F583E493FB744C
:10135A000193FA7402932FF9EA3EFA900011E4120B
:10136A0026F1905F8075F00CED122905EC75F00CF2
:10137A00A42583F583E493FB740193FA740293F929
:10138A00900476E0FEA3E0FF7C007D15122713E9A6
:10139A002FF9EA3EFA900012E41226F1900474E062
:1013AA00FCA3E0905F8075F00C122905EC75F00C37
:1013BA00A42583F583E493FB740193FA7402932FB3
:1013CA00F9EA3EFA90001374631226F1900477E06A
:1013DA00FFC007900474E0FEA3E0905F8075F00CF4
:1013EA00122905EE75F00CA42583F583E493FB74AA
:1013FA000193FA740293F9900476E0FE7C001227B6
:10140A0013E92FF9EA3EFA900014D0E01226F1907F
:10141A000477E004F07006900476E004F090047615
:10142A00E07004A3E064186003020CEB900475E01A
:10143A0004F07006900474E004F0900474E0700400
:10144A00A3E064026003020CE475625F7563809036
:10145A008000E49390116FF0D3940940037403F071
:10146A00126113D2AF126090125EAF123668123D4B
:0E147A00947F04124F48755501E49010B5F0B0
:10148800301A07C21A7F04124F48125158EF6009E8
:101498007E5F7F807D011239771251C0EF60097E2F
:1014A8005F7F8CE4FD12397730064490113CE0FCF4
:1014B800A3E0FDA3E0FEA3E0FFEF24FFFFEE34FF6F
:1014C800FEED34FFFDEC34FFFC90113C1228B79080
:1014D800113CE0FCA3E0FDA3E0FEA3E0FFEC4D4ED1
:1014E8004F700C90116EE0FF7D04125E8FC20612E1
:1014F80055BE900478EFF07003021BFBE014B4169D
:10150800004003021BF590151C75F003A4C5832544
:10151800F0C5837302155E02157F02164402171880
:101528000215AD02158C02159D0218D802198F02FA
:1015380019D9021942021A290217280217B00215EE
:10154800850218320218BC0218CA021BC9021BCD38
:10155800021BD4021BE490113CE0FCA3E0FDA3E0D5
:10156800FEA3E0FFEC4D4E4F7003021BF5C206A22E
:1015780002B39202021BF5126129021BF5C203C2D3
:10158800070218B6300006125E6F02198C125F3817
:10159800D20002198C300105125E6F8005125F3887
:1015A800D20102198C12607E30003685658285640E
:1015B80083C083C082E0FCA3E0FD7A007B01AE0417
:1015C8007802CEC313CE13D8F95401FFED54FBFDB6
:1015D800EF6B7E0054017802C333CE33CED8F98046
:1015E80037300147856582856483C083C082E0FC0B
:1015F800A3E0FD7A007B01AE047803CEC313CE13BB
:10160800D8F95401FFED54F7FDEF6B7E00540178D3
:1016180003C333CE33CED8F9FFEC4EFEED4FFFD0E7
:1016280082D083EEF0A3EFF002193C300506125E7B
:101638006F021BF5125F38D205021BF512607EE5BA
:1016480055700302170FE5652402FFE43564FAA913
:10165800077B01C001856582856483E013131354F9
:101668000325E0FFE433FE74A22FF9740C3EA801B1
:10167800FC7D01D0017E007F02122651856582859E
:101688006483C083C082E0FCA3E0FDEC1313135411
:1016980003FFEC54E7FCEF2401FFE433EF5403337A
:1016A800333354F84CFFEDD082D083CFF0A3EFF062
:1016B800856582856483E0FCA3E0FDEC1313135475
:1016C800036403700F856582856483EC54E7AF0576
:1016D800F0A3EFF0856582856483E0131313540348
:1016E80025E0FFE433FE74A22FF9740C3EFA7B0167
:1016F800E5652402FFE43564A807FC7D017E007FD0
:101708000212265102193C125F38755501021BF569
:10171800300F05125E6F8005125F38D20F02198CE8
:1017280012607E30087A856582856483C083C082B2
:10173800E0FCA3E0FDAE047807CEC313CE13D8F9BE
:101748005403FFEC54FEFCED547FFDEF2401FF7EB3
:1017580000EF54037807C333CE33CED8F9FFEC4EED
:10176800FEED4FFFD082D083EEF0A3EFF0856582C7
:10177800856483E0FCA3E0FDAE047807CEC313CEF6
:1017880013D8F9540364037012856582856483EC69
:1017980054FEFFED547FCFF0A3EFF0126175800384
:1017A800125F38D208021BF5300977125E6F90106D
:1017B800C2E014601F14601C14602F14602C1460A5
:1017C8004324057058856582856483C083C082E0A0
:1017D80054F9803D856582856483C083C082E05466
:1017E800F9FEA3E0FFEE44028014856582856483D8
:1017F800C083C082E054F9FEA3E0FFEE4404D08227
:10180800D0838015856582856483C083C082E04467
:1018180006FFA3E0D082D083CFF0A3EFF01261756A
:101828008003125F38D20902198C3007187E5F7F57
:1018380080EFB5630CEEB5620875625F75638C80E6
:10184800048E628F63856382856283740693F8E6EB
:1018580075F015A4FFE493FB740193FA7402932FB7
:10186800F9EA35F0FA900008122690D3940440075C
:10187800900008E41226F1856382856283740693DA
:10188800F8E675F015A4FFE493FB740193FA74026B
:10189800932FF9EA35F0FA900009122690D39404B0
:1018A8004007900009E41226F1C20312607E125B21
:1018B8008D021BF575625F756380125F38D2040272
:1018C800198C75625F75638C125F38D204021A2313
:1018D80012607E856582856483C083C082E0FEA332
:1018E800E0FF5401FBEF54FEFFEB6401FD5401FBE4
:1018F800EF4BFFD082D083EEF0A3EFF0ED7035858B
:101908006582856483C083C082E0FCA3E0FDECC3EC
:1019180013ED135401FFED54FDFDEF64015401254F
:10192800E0FFE433FEEC4EFEED4FFFD082D083EEB5
:10193800F0A3EFF0126175021BF530074785658249
:10194800856483C083C082E0FCA3E0FD7A007B014C
:10195800AE047806CEC313CE13D8F95401FFED5464
:10196800BFFDEF6B7E0054017806C333CE33CED86B
:10197800F9FFEC4EFEED4FFFD082D083EEF0A3EFDF
:10198800F0126175021A23300745856582856483E4
:10199800C083C082E0FCA3E0FDECC4F854F0C8EDBD
:1019A800C4540F485401FFED54EFFDEF6401540196
:1019B800C4F8540FC868FFE4C454F048FEEC4EFE67
:1019C800ED4FFFD082D083EEF0A3EFF01261758067
:1019D8004A300747856582856483C083C082E0FCFE
:1019E800A3E0FD7A007B01AE047805CEC313CE13C5
:1019F800D8F95401FFED54DFFDEF6B7E00540178F8
:101A080005C333CE33CED8F9FFEC4EFEED4FFFD0F1
:101A180082D083EEF0A3EFF012617512607E021B94
:101A2800F5200703021BF5200303021B989010B54D
:101A3800E06003021B8A856382856283740693F8DB
:101A4800E6FE9010B3E0FF6E7003021B829010B2A6
:101A5800E0FDEEB50508C203125FC6021BF58563FB
:101A680082856283E493FB740193FA740293F9907C
:101A780010B3E075F015A4F58285F083122807E508
:101A8800F05418FE856382856283740693F8E675C0
:101A9800F015A4F582E92582F9EA35F0FA1227DC77
:101AA800FDE5F054E74EFFEDCF8FF012283F856338
:101AB80082856283E493FB740193FA740293F9902C
:101AC80010B3E075F015A4F58285F083122807E5B8
:101AD800F05460FE856382856283740693F8E67528
:101AE800F015A4F582E92582F9EA35F0FA1227DC27
:101AF800FDE5F0549F4EFFEDCF8FF012283F856330
:101B080082856283E493FB740193FA740293F990DB
:101B180010B3E075F015A4FFE92FF9EA35F0FAE9FA
:101B28002402F9E43AFAC003C002C0018563828541
:101B38006283740693F8E675F015A4FFE493FB74CA
:101B48000193FA7402932FF9EA35F0FAE92402F9BD
:101B5800E43AA801FCAD03D001D002D0037E007F97
:101B680002122651856382856283740693F8E69093
:101B780010B2F07F04124F4880739010B57401F0D2
:101B8800806B9010B5E004F064047061C203805D5E
:101B9800D203C219C21BE5557003300F0DE4901033
:101BA800B5F09010B274FFF080069010B57401F093
:101BB800856382856283740693F8E69010B3F0809B
:101BC8002C7F0180027FFF125A0680219010B7A354
:101BD800E0FAA3E0F5828A837F01800E9010B7A314
:101BE800E0FAA3E0F5828A837FFF12293B12366868
:101BF800123D94125BBFEF7003021488901168E0E5
:101C08006431703590116EE0FF901169E06F7029B2
:101C18001260077F32125E0890116AE0FFA3E0FDB0
:101C2800A3E0FBA3E090047CF012349E7F32125EA6
:101C38000890116EE0FF125FF2901168E064327054
:101C48003590116EE0FF901169E06F7029126007FE
:101C58007F32125E0890116AE0FFA3E0FDA3E0FB6B
:101C6800A3E090047CF01237F77F32125E089011DF
:101C78006EE0FF125FF2901168E0642D702F9011F2
:101C88006EE0FF901169E06F70231260077F3212D7
:101C98005E0890116AE0FFA3E0FDA3E0FB1245E2B5
:101CA8007F32125E0890116EE0FF125FF2901168A9
:101CB800E0642E702F90116EE0FF901169E06F7054
:101CC800231260077F32125E0890116AE0FFA3E0DA
:101CD800FDA3E0FB1244217F32125E0890116EE0F2
:101CE800FF125FF2901168E0B41405D202123D941D
:101CF800901168E0B41505C202123D942002030257
:101D08001488901168E014602E24FD604224046059
:101D180003021488901169E0FFC3941E4003021463
:101D2800889008A5EFF0125088123668123D947F0B
:101D380005124F48021488901169E0FFC3941E40B1
:101D4800030214889008A5EFF01261960214887FA8
:0C1D58000F1257407F0F12560F02148824
:0F556D0075FFDE75FFAD75840F759601758C2087
:10557C00E4900479F0A3F090047AE004F0700690C3
:10558C000479E004F0900479E0B44EEBA3E0B4208D
:01559C00E628
:10559D00759701758A8843B73075EF06E4F5841267
:1055AD005F50125F1E12598E124ED412613302617A
:0155BD006E7F
:105F500075840F75A41175A57CE4F5A675A7E07589
:085F6000E12575E344F58422FC
:07616E00E4F58475D48422DE
:105F1E00E4F58443E60875DA3175DB3175DC3175ED
:0A5F2E00DD3175D983D2DEF584223F
:0A61330075E8C175BCF875D10322B0
:10609000751911751A70E4F513F5BB75E8D143E76E
:0260A0000222DA
:032A30000257CC7E
:1057CC00C0E0C083C082C0D075D000C006C2ED0559
:1057DC001AE51AAE197002051914F5828E83E5BF0D
:1057EC00F00513E513B40409751911751A707513C6
:1057FC00008513BB75E8D1D006D0D0D082D083D031
:02580C00E03288
:105DBE007F07125740901173E0FF125740901172F7
:105DCE00E0FF125740901171E0FF12574090117092
:055DDE00E0FF02574048
:105DE3007F0712560F901173E0FF12560F90117236
:105DF300E0FF12560F901171E0FF12560F901170D1
:055E0300E0FF02560F54
:104E5A0090047EEEF0A3EFF0F5828E83E493FB7468
:104E6A000193FA740293F99001F8122690D39405EB
:104E7A0040079001F8E41226F190047EE0FEA3E0D8
:104E8A00F5828E83A3A3A3740193FA740293F58225
:104E9A008A837F0112293B90047EE0FCA3E0FDF5A2
:104EAA00828C83E493FB740193FA740293F9900160
:104EBA00F8122690FF8D828C83A3A3A3740193FA20
:0A4ECA00740293F5828A8302293BEB
:1039770090047BEDF0900479EEF0A3EFF0F5828EE2
:1039870083740793F8E624FD7003023A1224FD704E
:1039970003023A1A24FA7003023A26147003023A11
:1039A70029147003023A2C240E6003023AEF9004A4
:1039B70079E0FEA3E0FFF5828E83740893FC740917
:0A39C70093F5828C83E024F8703B36
:1039D1008F828E83E493FB740193FA740293F990BE
:1039E10001F812269090047CF0E004F0B40502E4A2
:1039F100F090047CE0FD900479E0FEA3E0FF9001EB
:0B3A0100F8ED1226F1124E5A12613D42
:103A0C00123668023D94125B8D7F04024F4890047D
:103A1C007BE06003025DBE025DE302366802613D3D
:103A2C00E490047CF0900479E0FCA3E0FDF5828C3A
:103A3C0083740A93FE740B93F5828E83E075F015F4
:103A4C00A4FF8D828C83E493FB740193FA7402932C
:103A5C002FF9EA35F0FAE9240AF9E43AFA90047CF1
:103A6C00E07E0029F9EE3AFA12267790047DF06098
:103A7C00637F0312477590047CE0FF124775900436
:103A8C007DE014FF124775900479E0FCA3E0FDF58E
:103A9C00828C83740A93FE740B93F5828E83E0758B
:103AAC00F015A4FF8D828C83E493FB740193FA745C
:103ABC0002932FF9EA35F0FAE9240EF9E43AFA9078
:103ACC00047CE07E0029F9EE3AFA122677FF1247C1
:103ADC007512618390047CE004F0E0C394045003FD
:033AEC00023A316A
:013AEF0022B4
:0B61130090116FE090614693F5D322DD
:103C4E000001020408100000030418000000000028
:103C5E001F000000000018040300000000100804FC
:103C6E0002010000040A0A11110000010102021CE7
:103C7E0000001C02020101000010100808070000DD
:103C8E00070808101000008040C020A060E01090CF
:103C9E0050D030B070F0088848C828A868E8189846
:103CAE0058D838B878F8048444C424A464E414942E
:103CBE0054D434B474F40C8C4CCC2CAC6CEC1C9CE6
:103CCE005CDC3CBC7CFC028242C222A262E212920A
:103CDE0052D232B272F20A8A4ACA2AAA6AEA1A9AE6
:103CEE005ADA3ABA7AFA068646C626A666E61696CE
:103CFE0056D636B676F60E8E4ECE2EAE6EEE1E9E86
:103D0E005EDE3EBE7EFE018141C121A161E11191C7
:103D1E0051D131B171F1098949C929A969E91999B5
:103D2E0059D939B979F9058545C525A565E515959D
:103D3E0055D535B575F50D8D4DCD2DAD6DED1D9D55
:103D4E005DDD3DBD7DFD038343C323A363E3139379
:103D5E0053D333B373F30B8B4BCB2BAB6BEB1B9B55
:103D6E005BDB3BBB7BFB078747C727A767E717973D
:103D7E0057D737B777F70F8F4FCF2FAF6FEF1F9FF5
:063D8E005FDF3FBF7FFF75
:1060A2007F3812601C7F0612601C7D0EE4FF022AFC
:0160B20033BA
:10601C00900486EFF0125FDCEF20E7F9900486E045
:04602C00FF025AEA2B
:105FDC0075A0FFC2B6D2B5D2B77F14DFFEAFA0EF6B
:055FEC00903C9493FFBE
:015FF100228D
:0561AE007F0102601CEE
:105AEA00EF903C9493F5A07FFF7E00EF1F70011E9C
:105AFA00EF4E70F7C2B6C2B5D2B77E007FFFEF1F76
:105B0A0070011EEF4E70F7C2B77E007FFFEF1F7065
:065B1A00011EEF4E70F7C2
:015B20002262
:105B2100EF3395E0FE74942FF582743C3EF583E4E7
:105B310093F5A0C2B5D2B7D2B67FFF7E00EF1F703A
:105B4100011EEF4E70F7C2B77E007FFFEF1F70019D
:055B51001EEF4E70F78D
:015B5600222C
:0C2A3300901174E05FF04DFFF002601C99
:0E60D300AE07125FDCEF20E7F9AF06025B219B
:0859CB00E0FBA3E0FAA3E0F900
:1059D300900486EBF0A3EAF0A3E9F0900486E0FBE1
:1059E300A3E0FAA3E0F91226776017900486A3E4F4
:1059F30075F0011227C6A9F0FA122677FF1260D3B9
:035A030080D92225
:105BEF00900480EBF0A3EAF0A3E9F01261AEE4FDBC
:105BFF00FF1260EF9004801259CBE4FD7F01126019
:0E5C0F00EF9004831259CB7D117F010260EFEC
:0C60EF00EF75F040A42D2480FF02601C1F
:1060B3000001FF00FF000001010000FF00FF0100DD
:0960FB0044113C00000000C10644
:1052F400D295C296125E2BE4FCFDC004C005C00624
:10530400C007AFB0FEEF5403FFE4781012286FD04B
:1053140003D002D001D000EF4BFFEE4AFEED49FD71
:10532400EC488F598E588D57F5568F5F8E5E8D5D84
:10533400F55CAF80755A008F5BAF907560008F612C
:105344007B017A1179428B518A5289538A4F895051
:015354002236
:054D600090089AEFF03D
:104D6500E5502401FFE4354FFAA907A37401F0A328
:104D7500EAF0A3E9F090089BE0FBA3E0FAA3E0F9D1
:104D850074019011566B7008E965827003EA6583BA
:104D9500700D90089B04F0A37411F0A37442F09079
:104DA500089BE0FBA3E0FAA3E0F9E5518552838572
:104DB50053826B7008E965827003EA658360199018
:104DC500089AE0855082854F83F090089BA3E0FA0E
:084DD500A3E0AE028E4FF55081
:014DDD0022B3
:1055BE0053E6F7E5518552838553826401700AE5FF
:1055CE005065827004E54F65837003FF802FAB51E9
:1055DE000553E553AA527002055214F9122677FFAD
:1055EE0074019011566B700AE55365827004E55292
:1055FE006583700975510175521175534243E60862
:01560E002279
:105F68007E80E4FDEF5E24FF9292C293EEC313FE9F
:075F7800D2930DEDB408ED1A
:015F7F0022FF
:105E2B00D296E4FBC295ED25E0FDEC33FC309704F4
:105E3B00ED4401FDD2950BEBB410E9C296AF05AE64
:015E4B000452
:015E4C002233
:032A1E00021D6432
:101D6400C0E0C0F0C083C082C0D075D000C000C045
:101D740001C002C003C004C005C006C00720DF03C1
:031D8400022086B4
:101D8700E5126005D51202D21A125E2BE4FCFDC0E3
:101D970004C005C006C007AFB0FEEF5403FFE478E8
:101DA7001012286FD003D002D001D000EF4BF54DB1
:101DB700EE4AF54CED49F54BEC48F54AAF5FAE5EA0
:101DC700AD5DAC5CAB4DAA4CA94BF8C312285E6065
:101DD7003DE54D655FFFE54C655EFEE54B655DFDE9
:101DE700E54A655CFC9008961228B7900896E0FCD7
:101DF700A3E0FDA3E0FEA3E0FFEC4D4E4F600375AB
:101E07005403854D5F854C5E854B5D854A5CE55483
:101E170070030220841554E5546003022084E54DC5
:101E27005401FFE4FEFDFCFBFAF9F8C312285E70CB
:101E37000C90113C1228C30000AFC8D206E55965C3
:101E47004DFFE558654CFEE557654BFDE556654A80
:101E5700FC9008961228B7900896A3A3A3E0540114
:101E6700FFE4FEFDFCEF600DE54D5401FFEF60055B
:101E77007F01124D60900896A3A3A3E05402FFE4EC
:101E8700FEFDFCEF600DE54D5402FFEF60057F029C
:101E9700124D60900896A3A3A3E05404FFE4FEFD4F
:101EA700FCEF600DE54D5404FFEF60057F03124D15
:101EB70060900896A3A3A3E05408FFE4FEFDFCEF9F
:101EC700600DE54D5408FFEF60057F04124D6090EB
:101ED7000896A3A3A3E05410FFE4FEFDFCEF600DFA
:101EE700E54D5410FFEF60057F05124D6090089691
:101EF700A3A3A3E05420FFE4FEFDFCEF600DE54D36
:101F07005420FFEF60057F06124D60900896A3A34B
:101F1700A3E05440FFE4FEFDFCEF600DE54D5440A7
:101F2700FFEF60057F07124D60900896A3A3A3E01B
:101F37005480FFE4FEFDFCEF600DE54D5480FFEF9C
:101F470060057F08124D60900896A3A3E0FEEE544B
:101F570001FEE4FDFCEE600DE54C5401FEEE60056C
:101F67007F09124D60900896A3A3E0FEEE5402FE8F
:101F7700E4FDFCEE600DE54C5402FEEE60057F0AC1
:101F8700124D60900896A3A3E0FEEE5404FEE4FD14
:101F9700FCEE600DE54C5404FEEE60057F0B124D20
:101FA70060900896A3A3E0FEEE5408FEE4FDFCEE65
:101FB700600DE54C5408FEEE60057F0C124D6090F5
:101FC7000896A3A3E0FEEE5410FEE4FDFCEE600DC0
:101FD700E54C5410FEEE60057F0D124D609008969B
:101FE700A3A3E0FEEE5420FEE4FDFCEE600DE54CFD
:101FF7005420FEEE60057F0E124D60900896A3A355
:10200700E0FEEE5440FEE4FDFCEE600DE54C54406E
:10201700FEEE60057F0F124D60900896A3A3E0FEC9
:10202700EE5480FEE4FDFCEE600DE54C5480FEEEC0
:1020370060057F10124D60900896A3E0FDE4FEED69
:102047005401FDE4FCED600CE54B5401FD60057F98
:1020570011124D60900896A3E0FDE4FEED5402FDD9
:10206700E4FCED600CE54B5402FD60057F12124D58
:0F20770060854D59854C58854B57854A56C2DFB9
:0620860020D80330D967E9
:10208C00900896E580F0C2D9C2D8E0FFFDE55B6D03
:10209C0054C06053EFC413135403FDE55AC4F854F1
:1020AC00F0C8E55BC4540F487E00540CFFEF4D2480
:1020BC00B3F582EE3460F583E493FF900897F0A3B8
:1020CC00E54EF0EF254EF54EE0654E30E1109008F0
:1020DC0097E0B401047F1480027F13124D609008C6
:0720EC0096E0755A00F55B58
:0620F30020DA0330DB647B
:1020F900900896E590F0C2DBC2DAE0FDFFE5616F7A
:1021090054036050E561AE607802C333CE33CED854
:10211900F97E00540CFFED5403FDEF4D24B3F58215
:10212900EE3460F583E493FF900897F0A3E54EF051
:10213900EF254EF54EE0654E30E110900897E0B47A
:1021490001047F1580027F16124D60900896E07594
:042159006000F561CC
:10215D00D007D006D005D004D003D002D001D000D6
:0B216D00D0D0D082D083D0F0D0E03280
:103D9400E4FD3007353003057440FD800E3009041E
:103DA400ED4410FD300804ED4420FD30041C748003
:103DB400B56309745FB56204ED4480FD748CB5632A
:103DC40009745FB56204ED4408FDEDF4FF125F6809
:103DD400E4FD300772748CB56306745FB562010D3F
:103DE400856582856483E0FEA3E0FF30E004ED4452
:103DF40002FDEEC313EF1330E004ED4404FD8565CA
:103E040082856483E0FEA3E07806CEC313CE13D884
:103E1400F930E004ED4410FD856582856483E0FAA1
:103E2400A3E0FBAE027805CEC313CE13D8F930E07D
:103E340004ED4420FDEAC4F854F0C8EBC4540F4820
:103E440030E004ED4440FD300204ED4480FDEDF427
:103E5400FF125F68E4FD30076A200353E5556001F3
:103E64000D300F04ED4402FD200532300016856547
:103E740082856483E0FEA3E07802CEC313CE13D818
:103E8400F920E01930011A856582856483E0FEA378
:103E9400E07803CEC313CE13D8F930E004ED440424
:103EA400FD300004ED4408FD300104ED4410FD74C0
:103EB40080B56309745FB56204ED4440FDED448050
:0D3EC400FD8004ED4420FDEDF4FF025F6879
:104ED400E4F58475910575C80475C90875CBFF752B
:104EE400CAFC75CDFF75CCFC53877F759850438EF3
:104EF40010438920438840758DFE439802438748B8
:104F0400D2AC43E740758401759850F584438E1004
:104F140053890F438920438840758DFE858D8BD23C
:104F2400AC43E740F58453890F438920758DDF43F3
:104F34008E10758DE0858D8BD28E75840143E7408C
:044F4400E4F58422EA
:10595000E4F525F535F5367E027F4E8E458F468E71
:10596000418F42F525F533F5347E007F288E438F35
:10597000448E3D8F3E7E007F008E3B8F3C8E378F66
:0E598000387E007F148E3F8F408E398F3A2282
:032A0F000248C5B5
:1048C500C0E0C0F0C083C082C0D075D000C000C0B9
:0D48D50001C002C003C004C005C006C0073A
:1048E20075840030981DC2989008A0E599F0E0FF09
:1048F200125D729008A0E0B4080990089EE4F0A34B
:0C4902007407F0309942E534453360370B
:10490E00854482854383E09008A1F0C299F599050C
:10491E0030E5307002052FE534153470021533057D
:10492E0044E54470020543B44E12E543B4020D75DE
:05493E00430075442850
:074943008005C299754700D1
:10494A00D007D006D005D004D003D002D001D000C1
:0B495A00D0D0D082D083D0F0D0E0326B
:032A3F00024A0345
:104A0300C0E0C0F0C083C082C0D075D000C000C079
:0D4A130001C002C003C004C005C006C007FA
:104A2000758401309814C298AF99EFB408099008C2
:104A3000A2E4F0A37407F0125D98309942E5364580
:034A4000356037A7
:104A4300854682854583E09008A4F0C299F59905CF
:104A530032E53270020531E536153670021535053B
:104A630046E54670020545B47412E545B4040D7578
:054A7300450275464EEE
:0A4A78008005C2997548007584009E
:104A8200D007D006D005D004D003D002D001D00088
:0B4A9200D0D0D082D083D0F0D0E03232
:025D7200A9077F
:105D7400E5382401FFE43537FE7414B507097400CF
:105D8400B506047E007F00853882853783E9F08E6E
:035D9400378F380E
:015D970022E9
:025D9800A90759
:105D9A00E53A2401FFE43539FE7428B50709740091
:105DAA00B506047E007F14853A82853983E9F08E30
:035DBA00398F3AE4
:015DBD0022C3
:10574000E4F584E53464267004E533640260F4C251
:10575000AC053EE53EAC3D7002053D14F5828C8300
:10576000EFF0744EB53E0B7402B53D06753D007505
:105770003E280534E53470020533E547700575476A
:0657800001D299D2AC2217
:10560F0043E740E53664267004E535640260F475BF
:10561F00840153E7BF0542E542AC417002054114D6
:10562F00F5828C83EFF07474B5420B7404B54106A8
:10563F0075410275424E0536E53670020535E5486F
:0E564F007005754801D29943E740E4F58422C6
:10605800E538653C7004E537653B60047F018002E4
:036068007F002294
:10606B00E53A65407004E539653F60047F018002C5
:03607B007F002281
:105C1D00053CE53CAE3B7002053B14F5828E83E0FE
:105C2D00FFB40809900479E4F0A37407F07414B577
:0D5C3D003C0B7400B53B06753B00753C0048
:015C4A002237
:105C4B000540E540AE3F7002053F14F5828E83E0C0
:105C5B00FFB40809900479E4F0A37407F07428B535
:0D5C6B00400B7400B53F06753F00754014F6
:015C78002209
:032A0C000256ABC4
:1056AB00C0E0C0D075D000C004C005C006C007AFB5
:1056BB002AAE29AD28AC27EC4D4E4F6016EF24FFD8
:1056CB00F52AEE34FFF529ED34FFF528EC34FFF520
:1056DB0027800C752A80752996752898752700D018
:0C56EB0007D006D005D004D0D0D0E032AB
:102178004D6F6E6F00506F6C7900205057004166AC
:10218800740031006578745F41006578745F4200BF
:102198006578745F43006578745F440020202031BF
:1021A800006578744100657874420065787443006E
:1021B80065787444004320004323004420004423EE
:1021C8000045200046200046230047200047230002
:1021D8004120004123004220004356202564202549
:1021E8007300494E544552504F4C41544500696E56
:1021F800746572706F6C6174650025732078202592
:102208007300256425732E25642078202573002506
:1022180032642E253032642078202573004C6F6F8D
:1022280070436F756E746572203D202564004465A7
:102238006372656D656E74204C2E432E0053657471
:10224800204C2E432E203D202564004E6F204A75D9
:102258006D70004A756D70202B20256400436572EF
:102268007461696E7479203D2025642525004A75BE
:102278006D7020746F207374616765202564004A4F
:102288006D70546F20253264206966204C433E30BF
:10229800005374726F6265204120616464726573D3
:1022A80073005374616765202564005374726F620C
:1022B80065204220616464726573730046726565C7
:1022C8000050756C736500537573746E00456E61CC
:1022D800626C00312F333200312F323400312F310C
:1022E8003600312F313200332F333200312F38008E
:1022F800312F3600332F313600312F3400312F3350
:1023080000332F3800312F3200322F3300332F346F
:102318000077686F6C00332F320032004D756C7493
:10232800692054696D65202573002573202A2025AE
:1023380032642E25303264207365630054656D70F5
:102348006F20253364202A20257300436C6F636B4C
:10235800202A202573005374726F6265202563203C
:1023680061646472657373005374616765202573D3
:10237800002535752025357500436F70792054691F
:102388006D6520257300436F7069656400005374A0
:102398006167652025326420746F20253264004C03
:1023A800434420636F6E74726173743A25640053FA
:1023B800657474696E677320536176656400536150
:1023C80076652073657474696E67730053657474F9
:1023D800696E6773204C6F61646564004C6F61645B
:1023E8002073657474696E677300204142434445E5
:1023F800464748494A4B4C4D4E4F505152535455FD
:10240800565758595A6162636465666768696A6BAA
:102418006C6D6E6F707172737475767778797A30C7
:102428003132333435363738397E21402324255E1E
:10243800262A28292D2B3D7C0101FF52280104FF63
:1024480053550108FF5E4D0100FF52280108FF5E49
:102458004D0100FF53B50104FF53550108FF5E4DC0
:102468000104FF60300106FF5CD1010BFF5CFA013B
:102478000BFF5ECD0011FF2A0B0007FF5EE8010C81
:10248800FF5F03000EFF5EE8010CFF5F030107FF1B
:102498005EE80106FF618A0106FF61900103FF58AB
:1024A800D20108FF5A3F000BFF580E0108FF614E8A
:1024B800010BFF6156000BFF580E010CFF589100ED
:1024C8000BFF580E0108FF5A780014FF2A0B000D65
:1024D800FF60440000FF611E0000FF60E1414243CD
:1024E80044454647484A4B4C4D4E5000FF2178FF23
:1024F800217DFF2182FF2186FF218AFF218CFF2178
:1025080092FF2198FF219EFF21A4FF21A9FF21AE60
:10251800FF21B3FF21B8FF21BDFF21C0FF21C3FF69
:1025280021C6FF21C9FF21CCFF21CFFF21D2FF21E6
:10253800D5FF21D8FF21DBFF21DEFF22C4FF22C9FE
:10254800FF22CFFF22D5FF22DBFF22E0FF22E5FF9B
:1025580022EAFF22EFFF22F4FF22F8FF22FCFF23EA
:1025680001FF2305FF2309FF230DFF2311FF231577
:09257800FF2319FF231EFF23229B
:105EAF00E49010B6F09010C2F09010C0F09010BABD
:0E5EBF00F09010E2F0901106F09010E3F02247
:062A1200E49010BEF0226A
:104BCC0090048BEEF0A3EFF0AF051DEF7003024CD9
:104BDC006090048BE0FEA3E0F5828E83A3A3E493A4
:104BEC00FB740193FA740293F99010BEE0FF75F018
:104BFC0005A424C5F582E43410F583EBF0A3EAF0A8
:104C0C00A3E9F090048BE0FAA3E0FBF5828A83E43D
:104C1C0093FEEF75F005A424C3F582E43410F583FC
:104C2C00EEF08B828A83740193FF9010BEE075F0D6
:104C3C0005A424C4F582E43410F583EFF09010BE83
:104C4C00E004F090048CE02405F090048BE0340038
:054C5C00F0024BD42220
:104DDE009010BEE0FF60749010BBE0FBA3E0FAA35E
:104DEE00E0F9122677C39F4004E41226DF9010BB31
:104DFE00E0FBA3E0FAA3E0F9122677FE75F005A416
:104E0E0024C3F582E43410F583E0FFEE75F005A4BB
:104E1E0024C4F582E43410F583E0FD1260EF9010A7
:104E2E00BBE0FBA3E0FAA3E0F912267775F005A428
:104E3E0024C5F582E43410F583E0F9A3E0FAA3E08B
:0C4E4E009010B7C9F0A3EAF0A3E9F0222D
:105E6F009010BBE0FBA3E0FAA3E0F974011226BD8A
:105E7F00122677FF9010BEE0B50704E41226DF224A
:012A0A0022A9
:0F2A21009010B774FFF0A3742AF0A3740AF02288
:07551B00541FFF7B117A0011
:10552200900499EEF0A3EFF0AF05EF3395E0FEE0C3
:105532002FF0900499E03EF0E0FEA3E0FFBEFF0CE6
:10554200BFFF09E4900499F0A3F08016EFB50312AF
:10555200EEB5020EEB24FFFEEA34FF900499F0A3AD
:0B556200CEF0900499E0FEA3E0FF22D1
:1054C700856382856283E493FB740193FA74029384
:0F54D70024F9F9EA3401FA741CAD07900498F037
:1054E600900494EBF0A3EAF0A3E9F0900494E0FBB7
:1054F600A3E0FAA3E0F9122677FF7E00900498E075
:10550600FB7A00125522900494E0FBA3E0FAA3E094
:05551600F9EF0226DFA1
:10522800AC0730002EE5652404FFE43564FAA907CD
:105238007B01AD04900498740FF01254E6E56524E0
:1052480004F582E43564F583E0640A7036E5652484
:10525800068027E5652405FFE43564FAA9077B0184
:10526800AF04740F1254E0E5652405F582E4356453
:10527800F583E0B40A0DE5652407F582E43564F5A5
:0652880083E4F0026175F1
:1049650090048CEBF0A3EAF0A3E9F090048CE0FB53
:10497500A3E0FAA3E0F9122677B40A08900492E0BE
:1049850064016079900492E0FFA3E08FF0A4FF90AA
:10499500048FE0FBA3E0FAA3E0F9EF1226BD12268F
:1049A50077D3648094E34004749C804690048FE040
:1049B500FBA3E0FAA3E0F9122677C3648094805044
:1049C5003C90048CE0FBA3E0FAA3E0F91226777093
:1049D50014900493E0FF90048FE0FBA3E0FAA3E0BA
:1049E500F9EF0226BD90048FE0FBA3E0FAA3E0F9FE
:0E49F50074641226BD900492E0FF1252282234
:1053550090048BEFF0E5653000172404FFE4356415
:10536500FAA9077B01C003C002C001E565240680D8
:10537500152405FFE43564FAA9077B01C003C002C3
:10538500C001E5652407FFE43564FAA90790048F99
:10539500EBF0A3EAF0A3E9F090048BE0900492F01F
:1053A500A37401F0D001D002D003124965026175E2
:105E4D00E565300004240880022409FDE43564FA78
:105E5D00A9057B01AD079004987405F01254E60274
:025E6D0061755D
:1053B50090048BEFF0E5653000172404FFE43564B5
:1053C500FAA9077B01C003C002C001E56524068078
:1053D500152405FFE43564FAA9077B01C003C00263
:1053E500C001E5652407FFE43564FAA90790048F39
:1053F500EBF0A3EAF0A3E9F090048BE0900492F0BF
:10540500A3740AF0D001D002D00312496502617578
:106030007B007A007949AD079004987404F01254FB
:04604000E60261759E
:105CD10090048BEFF0E565240AFFE43564FE7C0057
:105CE100EF2549FFEC3EFAA9077B01E0FD900498FE
:095CF1007466F01254E6026175BC
:105CFA0090048BEFF0E565240EFFE43564FE7C002A
:105D0A00EF2549FFEC3EFAA9077B01E0FD900498D4
:095D1A007415F01254E6026175E3
:105ECD00E5652412FDE43564FAA9057B01AD079063
:0B5EDD0004987464F01254E602617532
:012A0B0022A8
:105EE800E5652414FDE43564FAA9057B01AD079046
:0B5EF80004987418F01254E602617563
:105F0300E5652413FDE43564FAA9057B01AD07902B
:0B5F130004987464F01254E6026175FB
:06618A001254C70261750A
:066190001254C702617504
:1058D200AD07856582856483A3A37E00A3E0540798
:1058E200FF7B057A00125522EF5407FF85658285FA
:1058F2006483A3A3C083C082E0FCA3E054F8FDEC60
:10590200FEED4FFFD082D083EEF0A3EFF00261757F
:105A3F00AD07856582856483A3A3E05407FEA3E0C9
:105A4F00FF7BE77A03125522EE5407FE85658285A8
:105A5F006483A3A3C083C082E054F84EFED082D0EB
:095A6F0083EEF0A3EFF002617573
:10580E00AD07856582856483E0C41354077E00541A
:10581E0003FF7B047A00125522EF5403C43354E085
:10582E00FE856582856483C083C082E0549FFCA39D
:10583E00E0FDEC4EFFEDD082D083CFF0A3EFF0026F
:02584E00617582
:1042380090048BEFF0A3EDF08FF0A4F085658285F4
:104248006483A3A3C083C082E0FCA3E0FD90048C38
:10425800E0F9FB3395E0FAEDAE047803CEC313CE54
:1042680013D8F9FFEE541FFE7C00ED5407FDEF2B29
:10427800FFEE3A541FFEEF7803C333CE33CED8F99E
:10428800FFEC4EFEED4FFFD082D083EEF0A3EFF0AF
:10429800E964017036856582856483A3A3E0FCA385
:1042A800E0FDAE047803CEC313CE13D8F9FFEE5465
:1042B8001FFEEF64014E7013856582856483A3A396
:1042C800ED54074410FFE4F0A3EFF08565828564A0
:1042D80083A3A3E0FCA3E0FDAE047803CEC313CE12
:1042E80013D8F9FFEE541FFED3EF94B8EE940B40A9
:1042F8003990048BE0D3648094804014856582856E
:104308006483A3A3ED5407FFEF44C0FF745D8016D8
:10431800856582856483A3A3C083C082A3E0540714
:0B432800FFD082D083E4F0A3EFF0226E
:08614E007D6412423802617504
:086156007D011242380261755F
:10589100AD07856582856483A3A3E0131313541FA9
:1058A1007E0012551BEF541F33333354F8FE8565C8
:1058B10082856483A3A3C083C082E05407FCA3E074
:1058C100FDEC4EFFEDD082D083CFF0A3EFF002616B
:0158D1007561
:105A7800AD07856582856483A3A37E00A3E01255E4
:105A88001BEF541FFF856582856483A3A3C083C071
:105A980082E0FCA3E054E0FDECFEED4FFFD082D0A5
:095AA80083EEF0A3EFF00261753A
:106044007B017A11796FAD079004987408F01254AB
:04605400E6026113EC
:0B611E00201B057F01125415D21B222C
:0E60E1002019081250887F04124F48D219224D
:08326D00900481EDF0A3EBF0E9
:10327500900484E0D39404400CA3E4F0A37407F015
:10328500E4900484F09010BB7401F0A37411F0A3D2
:103295007406F090048E74FFF0A37421F0A374E11A
:1032A500F07C003000047D0180027D02900491ECE9
:1032B500F0A3EDF0EF7BFF60067A2179EA80047ACE
:1032C5002179F6900493EBF0A3EAF0A3E9F07B01F2
:1032D5007A1079E4122AA7900481E0FFD3940A407A
:1032E5006990048E74FFF0A37422F0A37402F0EFCA
:1032F50075F003A424E2F582E43424F583E493F91C
:10330500740193FA740293900491C9F0A3EAF0A3AF
:10331500E9F0900484E075F003A42400F582E43418
:1033250025F583E493F9740193FA74029390049458
:10333500C9F0A3EAF0A3E9F07B017A1079F5122A26
:10334500A77E247F4F7D02023498900483E07003AA
:0333550002343B04
:10335800900481E075F064A4FFA3E07C002FFEECEC
:1033680035F0900487F0A3CEF0900487E0FAA3E04C
:10337800FB7D78FFAE02122725A3EFF0E075F07809
:10338800A4FFC3EB9FFFEA95F0FE7C007D0A12279D
:1033980025A3EFF090048E74FFF0A37422F0A374B9
:1033A8000AF0900489E0FEFD900491E4F0A3EDF0AA
:1033B800EF75F003A4241EF582E43425F583E49325
:1033C800F9740193FA740293900493C9F0A3EAF094
:1033D800A3E9F0EE75F078A4FFC3900488E09FFDA0
:1033E800900487E095F0FC90048AE075F00AA4FF49
:1033F800C3ED9FFEEC95F0900496F0A3CEF09004F8
:1034080084E075F003A42400F582E43425F583E410
:1034180093F9740193FA740293900498C9F0A3EA9B
:10342800F0A3E9F07B017A1079F5122AA77E247FB0
:01343800593A
:10343900805B90048E74FFF0A37422F0A37417F0DC
:10344900900481E0FF900491E4F0A3EFF0900482EE
:10345900E0FF900493E4F0A3EFF0900484E075F0AA
:1034690003A42400F582E43425F583E493F9740177
:1034790093FA740293900495C9F0A3EAF0A3E9F0D2
:103489007B017A1079F5122AA77E247F407D0312E9
:053499004BCC02607E37
:1060C3007480B56308745FB56203AF1722AF1822FB
:10481E009010BB7401F0A37410F0A374C0F012607A
:10482E00C3900491E4F0A3EFF090048E74FFF0A314
:10483E007422F0A37425F07B017A1079E4122AA772
:10484E00856582856483E0FEA3E07807CEC313CE30
:10485E0013D8F9540314600E14602424027055E426
:10486E009010F5F0804E90048E74FFF0A37422F039
:10487E00A37436F07B017A1079F5122AA780359051
:10488E00048E74FFF0A37422F0A37445F0E5652442
:10489E0012F582E43564F583E0FF900491E4F0A311
:1048AE00EFF07B017A1079F5122AA77E247F777DAF
:0748BE0001124BCC02607EE9
:103AF0009010BB7401F0A37410F0A374C2F07E2484
:103B00007F7C7D06124BCC856582856483E0C31380
:103B1000540314602A147003023B9D147003023B8B
:103B2000FA24036003023C4B90048E74FFF0A374EC
:103B300022F0A37453F07B017A1079E4023C4890A0
:103B4000048E74FFF0A37422F0A3745BF0E5652487
:103B500014F582E43564F583E02401FEE433900437
:103B600091F0A3CEF07B017A1079E4122AA7900499
:103B70008E74FFF0A37422F0A37465F0E56524133E
:103B8000F582E43564F583E02401FEE4339004918A
:103B9000F0A3CEF07B017A1079F5023C4890048EB8
:103BA00074FFF0A37422F0A37476F0E5652414F595
:103BB00082E43564F583E02401FEE433900491F05F
:103BC000A3CEF07B017A1079E4122AA790048E74B8
:103BD000FFF0A37422F0A37465F0E5652413F58269
:103BE000E43564F583E02401FEE433900491F0A30E
:103BF000CEF07B017A1079F5804E1260C39004916B
:103C0000E4F0A3EFF090048E74FFF0A37422F0A30D
:103C10007425F07B017A1079E4122AA790048E743F
:103C2000FFF0A37422F0A37487F0E5652414F582F5
:103C3000E43564F583E02401FEE433900491F0A3BD
:0E3C4000CEF07B017A1079F5122AA702607E81
:105020009010BB7401F0A37410F0A374B6F0900458
:105030008E74FFF0A37422F0A37499F07B017A10B0
:1050400079E4122AA790048E74FFF0A37422F0A3CF
:1050500074AAF0856382856283E493FB740193FAFA
:10506000740293F99001F91226902401FEE4339022
:105070000491F0A3CEF07B017A1079F5122AA77E75
:08508000247F9A7D01024BCC54
:104FB5009010BB7401F0A37410F0A374B6F09004C4
:104FC5008E74FFF0A37422F0A374B3F07B017A1002
:104FD50079E4122AA790048E74FFF0A37422F0A33B
:104FE50074AAF0856382856283E493FB740193FA66
:104FF500740293F99001F91226902401FEE433908E
:105005000491F0A3CEF07B017A1079F5122AA77EE0
:0B501500247F9F7D01124BCC02607EC7
:102DA70090048E74FFF0A37423F0A37424F0856558
:102DB70082856483E0C413540390254275F003129F
:102DC7002905E475F003A42583F583E493F97401D9
:102DD70093FA740293900491C9F0A3EAF0A3E9F07F
:102DE7007B017A1079E4122AA7856582856483E0DE
:102DF7001313135403147003022EE6147003022FE7
:102E0700A12402600302302F856582856483A3A312
:102E1700E0FEA3E07803CEC313CE13D8F9FFEE5438
:102E27001FFAAB077C007D64FE12277A900480EEC0
:102E3700F0A3EFF07C007D64122713C3EB9FFFEA3A
:102E47009EFE900480E07002A3E07007EF4E7003CF
:102E5700FE7F0190048E74FFF0A37423F0A37432F5
:102E6700F0856582856483A3A3A3E0540790250FAB
:102E770075F003122905E475F003A42583F583E4AF
:102E870093F9740193FA740293900491C9F0A3EA39
:102E9700F0A3E9F0900480E0FDA3E0900494CDF066
:102EA700A3EDF0A3EEF0A3EFF07B017A1079F51212
:102EB7002AA7E5559010BB60127401F0A37410F0B7
:102EC700A374BFF07E247FA4022F887401F0A3743B
:102ED70011F0A37407F07E247FAE7D0302302C85AA
:102EE7006582856483A3A3E0FEA3E0FF541FD39408
:102EF700E7E494034013856582856483A3A3EF54B5
:102F0700E04407FFEEF0A3EFF090048E74FFF0A308
:102F17007423F0A37444F0856582856483A3A3E0DA
:102F2700FCA3E0FDEC5407FEED2401FFE43E900412
:102F370091F0A3EFF0EC131313541F90254E75F087
:102F470003122905E475F003A42583F583E493F9B7
:102F5700740193FA740293900493C9F0A3EAF0A35F
:102F6700E9F07B017A1079F5122AA7E5559010BB95
:102F770060147401F0A37410F0A374BFF07E247F73
:102F8700A97D0102302C7401F0A37411F0A374071A
:102F9700F07E247FBD7D0202302C856582856483A7
:102FA700A3A3E0FEA3E0FF541FD39410E4940040D2
:102FB70013856582856483A3A3EF54E04410FFEE75
:102FC700F0A3EFF090048E74FFF0A37423F0A374C2
:102FD70053F0856582856483A3A3A3E0541F9025DE
:102FE7004E75F003122905E475F003A42583F583D4
:102FF700E493F9740193FA740293900491C9F0A3CE
:10300700EAF0A3E9F07B017A1079F5122AA7300FCD
:10301700179010BB7401F0A37411F0A37407F07E2E
:0B302700247FC77D02124BCC02607EAC
:104333009010BB7401F0A37410F0A374B6F0900452
:104343008E74FFF0A37423F0A3745EF07480B563DE
:1043530009745FB562047F4180027F42900491EF4C
:10436300F07B017A1079E4122AA785638285628340
:10437300E493FB740193FA740293F99001F9122602
:1043830090FFC39418501A90048E74FFF0A3742204
:10439300F0A374AAF0EF2401FEE433A3F0A3CE80CC
:1043A3006A856382856283E493FB740193FA7402E2
:1043B30093F99001F9122690D3941C40089001F9C7
:1043C30074181226F190048E74FFF0A37423F0A3E3
:1043D3007470F0856382856283E493FB740193FABE
:1043E300740293F99001F912269075F003A424BB8B
:1043F300F582E43424F583E493F9740193FA7402A7
:1044030093900491C9F0A3EAF0A3E9F07B017A1039
:0E44130079F5122AA77E247F9A7D01024BCCF8
:1046BE009010AAE0B52F28A3E0B53023A3E0B531C2
:1046CE001EA3E0B53219A3E0B52B14A3E0B52C0F51
:1046DE00A3E0652D7004A3E0652E7003024774906D
:1046EE00048E74FFF0A37423F0A37479F0A3E52B6A
:1046FE00F0A3E52CF0A3E52FF0A3E530F07B017AD3
:10470E001079E4122AA790048E74FFF0A37423F09C
:10471E00A37479F0A3E52DF0A3E52EF0A3E531F017
:10472E00A3E532F07B017A1079F5122AA79010AA30
:10473E00E52FF0A3E530F0A3E531F0A3E532F0A3C9
:10474E00E52BF0A3E52CF0A3E52DF0A3E52EF090DC
:10475E0004837401F0A37410F0A374F5F07B017A56
:06476E001079E4125BEF7C
:014774002222
:105F98009010BB7401F0A37410F0A374C1F07E24B8
:075FA8007FD17D01024BCC0B
:103ED100856382856283E493FB740193FA74029390
:103EE100F9740693F8E675F015A4F58285F083124E
:103EF1002807E5F01313135403FD9010B3E075F098
:103F010015A4F58285F083122807E5F013131354E5
:103F1100036D7001E4704485638285628393FB7451
:103F21000193FA740293F9740693F8E675F015A4F7
:103F3100F58285F083122807E5F0C4135403FD9040
:103F410010B3E075F015A4F58285F083122807E51A
:0E3F5100F0C41354036D7001E460037F00227E
:103F5F00856382856283740693F8E675F015A4FF76
:103F6F00E493FB740193FA7402932FF9EA35F0FA94
:103F7F00E92402F9E43AFA900480EBF0A3EAF0A303
:103F8F00E9F0856382856283E493FB740193FA748D
:103F9F000293F99010B3E075F015A4FFE92FF9EA39
:103FAF0035F0FAE92402F9E43AFA900483EBF0A32E
:103FBF00EAF0A3E9F0A37402F0900486E0FF14F096
:103FCF00EF602D900483E0FBA3E475F0011227C688
:103FDF00A9F0FA122677FF900480E0FBA3E475F0B6
:103FEF00011227C6A9F0FA1226776F60CC7F002244
:033FFF007F01221D
:104002009010BB7401F0A37410F0A374B4F090107C
:10401200B5E01470030240A61470030240D314707A
:10402200030240FD2403600302412A123ED1EF7BCA
:10403200FF60067A23798E80047A23799590049121
:10404200EBF0A3EAF0A3E9F090048E74FFF0A374FE
:1040520023F0A37481F07B017A1079E4122AA790ED
:10406200048E74FFF0A37423F0A37496F09010B33F
:10407200E02401FEE433900491F0A3CEF085638244
:10408200856283740693F8E62401FEE43390049378
:10409200F0A3CEF07B017A1079F5122AA77E247F55
:1040A200D102412590048E74FFF0A37423F0A3740F
:1040B200A7F090116FE02401FEE433900491F0A385
:1040C200CEF07B017A1079E4122AA77E247FD68073
:1040D2005290048E74FF301B0AF0A37423F0A37471
:1040E200B78008F0A37423F0A374C6F07B017A10A2
:1040F20079E4122AA77E247FDB802890048E74FF45
:1041020030190AF0A37423F0A374D48008F0A374C6
:1041120023F0A374E4F07B017A1079E4122AA77EDB
:09412200247FE07D01124BCC2248
:10366800E5652408F582E43564F583E0D3940440E5
:103678000990047EE4F0A37407F0E5652409F58257
:10368800E43564F583E0D39404400990047EE4F0C3
:10369800A37407F0122A12E49010F5F09010E4F0E9
:1036A8002007030237DA3003061240020237DD3002
:1036B800003D856582856483A3E05401FFC007E56A
:1036C800652404F582E43564F583E0FDE5652406A8
:1036D800F582E43564F583E0FB856582856483E0E3
:1036E800FEA3E07802CEC313CE13D8F9023789308F
:1036F800014A856582856483E0C313A3E0135401FE
:10370800FFC007E5652405F582E43564F583E0FD2F
:10371800E5652407F582E43564F583E0FB85658279
:10372800856483E0FEA3E07803CEC313CE13D8F9F3
:103738005401900483F0E5652409804F30055F202B
:103748000005200102D200856582856483A3E054C8
:1037580001FFC007E5652404F582E43564F583E0DC
:10376800FDE5652406F582E43564F583E0FB8565AF
:1037780082856483E0FEA3E07802CEC313CE13D81B
:10378800F95401900483F0E5652408F582E4356472
:10379800F583E0900484F0D00712326D803730084A
:1037A8000512481E802F300905123AF08027300C88
:1037B80005125020801F300D05124FB58017E555B2
:1037C8007003300F05122DA7800B30040812433305
:1037D8008003125F989004837401F0A37410F0A31F
:0F37E80074F5F07B017A1079E4125BEF024DDE8D
:017FFF00AFD2
:0554150090048BEFF094
:10541A0012615E7E807F0090116FE0FD124B369024
:10542A008000E49390048CF0E4F090048BE0FFA3F6
:10543A00E0FEC39F502C75F0FCEEA42401F582E532
:10544A00F03480F583EE75F003A42583AF82FE7CE9
:10545A00087DA67BFC7A0312578690048CE004F040
:05546A0080C8025C791E
:10412B007B017A0879A690047F1228C3000003FC58
:10413B00E4FD125D23E4FFE4FEE4FD75F0FEEFA465
:10414B0024B4F582E5F03408F5832FF58375F0156B
:10415B00EE122905E5822DF582E43583F583740A89
:10416B00F00DEDB404D575F0FEEFA424A8F582E5AF
:10417B00F03408F5832FF58375F015EE122905C081
:10418B0083C082A3E05407FDED4420FDD082D08391
:10419B007403F0A3EDF075F0FEEFA424B9F582E5FE
:1041AB00F03408F5832FF58375F015EE122905749D
:1041BB0063F075F0FEEFA424AEF582E5F03408F55C
:1041CB00832FF58375F015EE122905E4F075F0FEDB
:1041DB00EFA424AFF582E5F03408F5832FF5837552
:1041EB00F015EE122905E4F075F0FEEFA4249EF510
:1041FB0082E5F0340AF5832FF583E4F075F0FEEFDA
:10420B00A4249FF582E5F0340AF5832FF583E4F0BF
:10421B000EEE641860030241440FEF640260030268
:0D422B00414290116F7405F07F1E02541582
:09613D00201E03126166D21E222D
:0761750012613D75121422B6
:10546F00907FFFE493601812412B900479747FF0C2
:10547F00A374FFF07E7FFFE4FD124B36125C797B45
:10548F00017A0C79A290047F1228C300000006E471
:10549F00FD125D23E49008A5F0900CA4E054F8FEF3
:1054AF00743BFF900CA4EEF0A3EFF0EE54074470A2
:0754BF00900CA4F0A3EFF034
:0154C60022C3
:1050880090048B74FAF09008A5E0FF7E007C037D05
:10509800FC12271374012FF974803EFA7BFF78A65F
:1050A8007C087D017E037FFC1226519008AEE0D378
:1050B8009404900A9EE090048BF0D394054005E494
:1050C800900A9EF0900C9CE0D394054002E4F09086
:1050D8000A9FE0D3941C4002E4F0900C9DE0D39426
:0750E8001C4002E4F0C21EAF
:0150EF00229E
:10295D007FFA12615E9008A5E0FF75F0FEA4249E3B
:10296D00F582E5F0340AF583EF2583F583E0D39402
:10297D0005401C9004797407F075F0FEEFA4249EB9
:10298D00F582E5F0340AF583EF2583F583E4F090C5
:10299D0008A5E0FF75F0FEA4249FF582E5F0340A4A
:1029AD00F583EF2583F583E0D3941C401C900479C7
:1029BD007407F075F0FEEFA4249FF582E5F0340A5C
:1029CD00F583EF2583F583E4F0908000E493900484
:1029DD0079F09008A5E0FF75F0FCA42401F582E5DF
:1029ED00F03480F583EF75F003A42583AF82FE7C70
:0D29FD00087DA67BFC7A03125786025C79E8
:0661960012295DC21E2269
:07617C00301F03126196229F
:032A1B00025088DE
:104A9D00901160EBF0A3EAF0A3E9F0A3ECF0A3ED25
:014AAD00F018
:104AAE0090116374FFF5F01227C645F060719011F6
:104ABE0060E0FBA3E475F0011227C6A9F0FA1226F6
:104ACE0077FD3395E0FC901165E0FFEF6DFDA3E0FF
:104ADE00F8E4F0E8901165F0ECC4F854F0C868FE04
:104AEE00EDC4540F48FFEE6CFEEF6DFFE06EF0A3C9
:104AFE00E06FF0EF7805C333CE33CED8F9FF9011C7
:104B0E0065E06EF0A3E06FF0EF7807C333CE33CEDF
:104B1E00D8F9FF901165E06EF0A3E06FF080819000
:074B2E001165E0FEA3E0FFAA
:014B3500225D
:054F480090048BEFF066
:104F4D00A37401F0A37408F0A374A6F0A37401F088
:104F5D00A3740AF0A374A4F0A37401F0A374FEF07B
:104F6D0012574090048BE0803890049274FFF5F056
:104F7D001227C645F0603090048CE0FBA3E475F079
:104F8D00011227C6A9F0FA122677FF125740900496
:104F9D008FE0FBA3E475F0011227C6A9F0FA1226E3
:074FAD0077FF12560F80C2CE
:014FB40022DA
:0A349E0090047AEDF0900479EFF04D
:1034A800D39B5003023589E024FFFEE434FF9004E7
:1034B8007EF0A3CEF0EB1490047DF090047AE02423
:1034C800FFFFE434FFFE90047EE0FCA3E0FDD39F01
:1034D800EE6480F8EC6480984003023667908001BF
:1034E80075F0FCED122905EC75F0FCA42583F8EDC8
:1034F80075F003A428AF82900485F0A3EFF0900440
:103508007DE0FF7E007C037DFC12271374012FF9F8
:1035180074803EFA90048274FFF0A3EAF0A3E9F005
:10352800E4900480F0A3F0900482A3E475F0011203
:1035380027C6FEAFF0900485E475F0011227C68512
:10354800F082F583E493FD124B36900481E004F099
:103558007006900480E004F0C3900481E094FC902D
:103568000480E0940340C0125C7990047FE004F08A
:10357800700690047EE004F090047DE004F00234CC
:10358800C390047AE024FFFEE434FF90047EF0A3A5
:10359800CEF090047CE014A3F0900479E024FFFFBF
:1035A800E434FFFE90047EE0FCA3E0FDC39FEE64DC
:1035B80080F8EC648098500302366790800175F0BB
:1035C800FCED122905EC75F0FCA42583F8ED75F0E7
:1035D80003A428AF82900485F0A3EFF090047DE067
:1035E800FF7E007C037DFC12271374012FF9748081
:1035F8003EFA90048274FFF0A3EAF0A3E9F0E490A5
:103608000480F0A3F0900482A3E475F0011227C6A9
:10361800FEAFF0900485E475F0011227C685F082AC
:10362800F583E493FD124B36900481E004F07006B4
:10363800900480E004F0C3900481E094FC9004803E
:10364800E0940340C0125C7990047FE024FFF0907E
:0F365800047EE034FFF090047DE014F00235A111
:013667002240
:0537F70090047AEDF0E2
:1037FC00EF1490087EF0EB14A3F090047AE014FF21
:10380C0090087EE0D39F4003023976A3E0FF75F069
:10381C00FCA42401F582E5F03480F583EF75F00308
:10382C00A42583AF82FEE4900880F0A3F09008807A
:10383C00E0FCA3E0FDC394FCEC9403502B0FEFAA27
:10384C000670010E14F5828A83E493FB74822DF5C5
:10385C008274043CF583EBF0900881E004F070CDA9
:10386C00900880E004F080C590087FE0FF7E007C2B
:10387C00037DFC12271374012FF974803EFA900417
:10388C007D74FFF0A3EAF0A3E9F090087EE0FF75E9
:10389C00F0FCA42401F582E5F03480F583EF75F09B
:1038AC0003A42583AF82900480F0A3EFF0E490088A
:1038BC0080F0A3F090047DA3E475F0011227C6FEFE
:1038CC00AFF0900480E475F0011227C685F082F504
:1038DC0083E493FD124B36900881E004F07006905F
:1038EC000880E004F0C3900881E094FC900880E02C
:1038FC00940340C090087EE0FF7E007C037DFC12A8
:10390C00271374012FF974803EFA90047D74FFF034
:10391C00A3EAF0A3E9F0E4900880F0A3F09008800B
:10392C00E0FCA3E0FDC394FCEC9403502D90047DCB
:10393C00A3E475F0011227C6FEAFF074822DF58258
:10394C0074043CF583E0FD124B36900881E004F0E2
:10395C0070CB900880E004F080C3125C7990087EF4
:0A396C00E004F0A3E004F0023806C6
:01397600222E
:07442100900479EBF0AC07F9
:10442800A3E5C1F0A2AFE433A3F0AF05A3E4F0A382
:10443800EFF0E07F00FE90047CF0A3EFF0AD04ED18
:10444800FF90047CEEF0A3EFF0C2AF43C15D90088B
:10445800A5740FF012615E9008A5E0FF7E007C0352
:104468007DFC12271374012FF974803EFA900480A2
:1044780074FFF0A3EAF0A3E9F0E490047EF0A3F05F
:1044880090047DE0FF90047CE0FD900479E0FBE47B
:10449800900491F0D210124504900483EFF0FD903F
:1044A8000480A3E475F0011227C6FEAFF0124B3664
:1044B80090047DE004F0700690047CE004F0900421
:1044C8007FE004F0700690047EE004F0C390047F5F
:1044D800E094FC90047EE0940340A5125C79900877
:1044E800A5E004F0E0C3941E500302445C90047AF3
:0C44F800E0F5C1A3E024FF92AF02618355
:0745E200900479EBF0AC0737
:1045E900A3E5C1F0A2AFE433A3F0AF0590047EE4E4
:1045F900F0A3EFF0E07F00FE90047EF0A3EFF0ADB2
:1046090004EDFF90047EEEF0A3EFF0C2AF43C15D6D
:104619009008A5740FF09008A5E0FFC3941E40030D
:104629000246AF75F0FCEFA42401F582E5F0348071
:10463900F583EF75F003A42583AF82900480F0A37E
:10464900EFF0E490047CF0A3F090047FE0FF900485
:104659007EE0FD900479E0FB900480E475F001129E
:1046690027C685F082F583E493900491F0C2101275
:10467900450490047FE004F0700690047EE004F0A5
:1046890090047DE004F0700690047CE004F0C3908F
:10469900047DE094FC90047CE0940340AC9008A570
:1046A900E004F002461F90047AE0F5C1A3E024FF7C
:0546B90092AF026183D5
:10528E0090088AE584F0A2AF9210AF01AE027C00C6
:10529E00E4FDA31228B7D390088EE0940090088DF9
:1052AE00E09470402CE0FEA3E07866A60608F6E4D3
:1052BE00F584C2AF43B701758F0318E6FE08E6F515
:1052CE00828E83E4F0F58F53B7FE90088904F08048
:1052DE0005E4900889F0A21092AF90088AE0F58458
:0552EE00900889E0FFBB
:0152F3002298
:054CE10090088FEDF0CA
:104CE600900891E584F0A2AF9210AF01AE027C006D
:104CF600E4FDA31228B7D3900895E0940090089499
:104D0600E09470404090088FE0FFFD3395E0FCEDA5
:104D1600F44C6029900894E0FCA3E07866A60408A9
:104D2600F6E4F584C2AF43B701758F0118E6FC08B7
:104D3600E6F5828C83EFF0E4F58F53B7FE9008908A
:104D46007401F08005E4900890F0A21092AF9008EC
:094D560091E0F584900890E0FF63
:014D5F002231
:1050F000900889EEF0A3EFF0A3ECF0A3EDF0A3EAA3
:10510000F0A3EBF090088DE07002A3E060499008F6
:1051100089E0FEA3E0AA06F97B01A3E0FEA3E0F587
:10512000828E83E0FD124CE1EF602C90088EE0242B
:10513000FFF090088DE034FFF090088CE004F070F0
:105140000690088BE004F090088AE004F070B590B7
:085150000889E004F080AD22A3
:08615E00E4900CA8F0A3F0226C
:105C7900900CA8E0FEA3E0AA06F97B0112528EEF70
:105C89006012900CA8E0FEA3E0FF7C0C7DAA1B7AB1
:0C5C9900041250F0E4900CA8F0A3F022DC
:0D4B3600900884EDF0900882EEF0A3EFF0FF
:104B4300EE54FCFE900CA8E0FCA3E0FD7002EE6CBA
:104B53006059ED4C6003125C79900882E0FEEE54DC
:104B6300FCFE7F00900CA8F0A3EFF0900885EEF018
:104B7300A3EFF0A3740CF0A374AAF07FFF7E03905D
:104B83000885E475F0011227C685F082F583E49366
:104B9300FD900887E475F0011227C685F082F5833E
:104BA300EDF0EF1F70011EEF4E70D4900884E0FF0C
:104BB300900882E0FCA3E0FDEC5403FC74AA2DF5FD
:084BC30082740C3CF583EFF055
:014BCB0022C7
:1057860090048DEEF0A3EFF0A3ECF0A3EDF0A3EA06
:10579600F0A3EBF090049174FFF5F01227C645F0E4
:1057A600602390048DE475F0011227C6AFF0FE90D9
:1057B600048FE475F0011227C685F082F583E0FDBB
:0657C600124B3680CF22D9
:055D230090047EEDF08C
:105D2800AF01AB0790047F74FF122884EC4D4E4FEF
:105D3800601090047EE08B828A83F00BBB00010A1E
:025D480080E2F7
:015D4A002236
:105FAF00E4FD0FEFAA0670010E14F5828A83E060FC
:065FBF00030D80EEAF05AA
:015FC50022B9
:10565D00901158EBF0A3EAF0A3E9F090115E74FFFE
:10566D00F5F01227C645F0603490115BE0FBA3E026
:10567D00FAA3E0F9122677FF901158E0FBA3E0FAA8
:10568D00A3E0F9EF1226DF901159E475F00112270E
:0E569D00B090115CE475F0011227B080BE22BF
:105E8F00900479EFF0A3EDF07F0A12477590047933
:105E9F00E0FF12477590047AE0FF124775026183A5
:086166007F02124775026183FC
:065BBF001261A2EF602755
:105BC5009004797411F0A37467F0125B579004790F
:105BD500E475F0011227C685F082F583EFF01261B6
:075BE500A8EF70E67F01222A
:035BEC007F002215
:105FF200900479EFF07F2F124775900479E0FF1239
:056002004775026183F7
:10600700900479EFF07F30124775900479E0FF1222
:056017004775026183E2
:104C610001011140010000000000000000000000EF
:104C71000000000000000000000000000000000033
:104C81000000000000000000000000000000000023
:104C91000100001704010AA00101115600000000E3
:104CA10001011141010000000000000000000000AE
:104CB10000000000000000000000000000000000F3
:104CC10000000000000000000000000000000000E3
:104CD1000100001804010C9E0101115700000000A1
:06619C00E4F50FF50E22F0
:10515800126058EF605FE50E601F150EE509450AFD
:10516800604C125C1DAB08050AE50AAA0970020525
:105178000914F9EF1226DF8035125C1D8F10EF2518
:10518800E025E02461F582E4344CF583E493F50EE0
:10519800EF25E025E02462F582E4344CF583E493BE
:1051A800FB740193FA7402938B088A09F50AE50ED9
:0851B80070037F01227F002239
:1051C00012606BEF605FE50F601F150FE50C450D7A
:1051D000604C125C4BAB0B050DE50DAA0C70020583
:1051E0000C14F9EF1226DF8035125C4B8F11EF257E
:1051F000E025E024A1F582E4344CF583E493F50F37
:10520000EF25E025E024A2F582E4344CF583E49315
:10521000FB740193FA7402938B0B8A0CF50DE50F66
:0852200070037F01227F0022D0
:105F80000108A6FF5740151011401156010AA4FF41
:085F9000560F161111411157C3
:03000000020C00EF
:03000300022A03CB
:03000B00022A06C0
:03001300022A09B5
:03001B00022A0CAA
:03002300022A0F9F
:03002B00022A1294
:03003300022A1589
:03003B00022A187E
:03004300022A1B73
:03004B00022A1E68
:03005300022A215D
:03005B00022A2452
:03006300022A2747
:03006B00022A2A3C
:03007300022A2D31
:03007B00022A3026
:03008300022A331B
:03008B00022A3610
:03009300022A3905
:03009B00022A3CFA
:0300A300022A3FEF
:100C0000787FE4F6D8FD9000007F007E20E4F0A31A
:0A0C1000DFFCDEFA758167020C5567
:02610400C121B7
:0C61070075C04475CFE2C2C375C303220B
:10598E007E117F1490110CEEF0A3EFF0901110EE3B
:10599E00F0A3EFF0901108EEF0A3EFF07E117F2848
:1059AE0090110EEEF0A3EFF0901112EEF0A3EFF0C7
:0D59BE0090110AEEF0A3EFF0C22002610785
:105AB100901110E475F0011227C685F082F583EF8D
:105AC100F0901110E475F0011227C685F082F5837C
:105AD100EDF0901110E0B4110FA3E0B4280A901179
:095AE100107411F0A37414F022FA
:07618300C220C2C4D2C522F4
:10477500202055D220901112E475F0011227C6852C
:10478500F082F58374FFF07C117D3C901112E0B549
:10479500040FA3E0B5050A9011127411F0A3742853
:1047A500F0901112E475F0011227C685F082F583A9
:1047B500E4F0901112E0B5040FA3E0B5050A9011DD
:1047C500127411F0A37428F0901112E475F001121F
:1047D50027C685F082F583E4F0901112E0B4110F3D
:1047E500A3E0B43C0A9011127411F0A37428F09060
:1047F5001112E475F0011227C685F082F583EFF0FA
:10480500901112E0B4110FA3E0B43C0A9011127498
:0948150011F0A37428F07F0122C8
:105CA50090110CE0FCA3E0FD901108E0B50408A3F9
:105CB500E0B505037F002290110CE0FCA3E0F5821E
:0C5CC5008C83E0B507037F01227F0022E2
:105B570090110DE004F0700690110CE004F0901124
:105B67000CE475F0011227C685F082F583E0FF90FB
:105B7700110CE0B4110FA3E0B4280A90110C7411B2
:055B8700F0A37414F00E
:015B8C0022F6
:0661A2007FFF125CA52244
:0661A800E4FF125CA522D9
:032A180002303257
:10303200C0E0C0F0C083C082C0D075D000C000C064
:1030420004C005C006C007E5C154F812291132298F
:1030520000308D08308D1030DB18312720313428B4
:1030620031BF3031CB3831DC5031DC5831EF603197
:10307200DE6831EF7031DE7831DC8031FE8831DCA0
:103082009031FE983211A000003256C2C590110B49
:10309200E004F0700690110AE004F07E117F3C908B
:1030A200110AE0B5060FA3E0B5070A90110A7411E0
:1030B200F0A37428F090110AE475F0011227C68576
:1030C200F082F583E0F5C290110AE06E7003A3E08E
:1030D2006F60030232560231B290110BE004F070BD
:1030E2000690110AE004F07E117F3C90110AE0B5CF
:1030F200060FA3E0B5070A90110A7411F0A3742811
:10310200F090110AE475F0011227C685F082F5836A
:10311200E0F5C290110AE06E7003A3E06F60030253
:1031220032560231B290110EE0FFA3E090110ACFA5
:10313200801B901112E0FEA3E0FF90110AE0FCA3B5
:10314200E0FDB50713ECB5060F90110EEEF0A3EFFC
:10315200F0C2C5D2C40232568D828C83E0B4FF071E
:10316200C2C4D2C502325690110BE004F070069030
:10317200110AE004F07E117F3C90110AE0B5060FBF
:10318200A3E0B5070A90110A7411F0A37428F09015
:10319200110AE475F0011227C685F082F583E0F585
:1031A200C290110AE06E7003A3E06F600302325610
:1031B20090110A7411F0A37428F002325690110E85
:1031C200E0FFA3E090110A803D90110EE0FFA3E022
:1031D20090110ACFF0A3EFF0807A801790110EE0E1
:1031E200FFA3E090110ACFF0A3EFF0D221ADC27F8E
:1031F200FF8004ADC2E4FF125AB18058901108E07A
:10320200FFA3E0901110CFF0A3EFF0D2C48045905D
:103212001110E0FFA3E0901108CFF0A3EFF03021EE
:1032220033D2C5C221802D90110EE0FEA3E0FF90A3
:10323200110AEEF0A3EFF0901108E0FDA3E0901167
:1032420010CDF0A3EDF0D2C4A3E06E7003A3E06F43
:103252006002D2C5C2C3D007D006D005D004D000C8
:0B326200D0D0D082D083D0F0D0E0327A
:0745040090048EEFF0A90501
:10450B00C21120C3FD20C5FAC2C4D2C5E4FFFD30E1
:10451B00C3FD30C3FDE5C154F8FC64086004ECB482
:10452B001013EFB40105EB44018003EB54FEF5C20D
:10453B007D010245D0ECB4180B89C27D02C2C4C206
:10454B00C50245D0ECB420028045EC6428703CEDEC
:10455B00B4020E90048EE0F5C27D03C2C5C2C480C6
:10456B0064EDB4031B301008D2C57F01C2C4805563
:10457B00900491E0F5C2C2C57D04E4FFC2C480453E
:10458B00ED64047040D2C47D05803AECB4300AD29D
:10459B00C4D2C57D08E4FF802CECB438028022EC39
:1045AB00B44006C2C2C2C5801CECB448028012ECF7
:1045BB00B450028004ECB45808D2C47D07AEC2805C
:1045CB0004D2C4D2C5C2C3ED64076008ED640560B4
:0645DB000302451DAF06BE
:0145E10022B7
:100C1A00020C9AE493A3F8E493A34003F68001F24A
:100C2A0008DFF48029E493A3F85407240CC8C333DB
:100C3A00C4540F4420C8834004F456800146F6DFAA
:100C4A00E4800B01020408102040809060FBE47EDF
:100C5A00019360BCA3FF543F30E509541FFEE4939F
:100C6A00A360010ECF54C025E060A840B8E493A366
:100C7A00FAE493A3F8E493A3C8C582C8CAC583CA91
:100C8A00F0A3C8C582C8CAC583CADFE9DEE780BE49
:016106000098
:10258100E709F608DFFA8046E709F208DFFA803E3C
:1025910088828C83E709F0A3DFFA8032E309F60829
:1025A100DFFA8078E309F208DFFA807088828C8391
:1025B100E309F0A3DFFA806489828A83E0A3F60845
:1025C100DFFA805889828A83E0A3F208DFFA804C1F
:1025D10080D280FA80C680D4806980F280338010F6
:1025E10080A680EA809A80A880DA80E280CA80335F
:1025F10089828A83ECFAE493A3C8C582C8CCC583D7
:10260100CCF0A3C8C582C8CCC583CCDFE9DEE780A6
:102611000D89828A83E493A3F608DFF9ECFAA9F025
:10262100EDFB2289828A83ECFAE0A3C8C582C8CC7B
:10263100C583CCF0A3C8C582C8CCC583CCDFEADE94
:10264100E880DB89828A83E493A3F208DFF980CCF6
:1026510088F0EF60010E4E60C388F0ED2402B404EF
:102661000050B9F582EB2402B4040050AF23234596
:0626710082239025D173C5
:10267700BB010689828A83E0225002E722BBFE0261
:09268700E32289828A83E4932294
:10269000BB010CE58229F582E5833AF583E02250FF
:1026A00006E92582F8E622BBFE06E92582F8E22249
:0D26B000E58229F582E5833AF583E4932263
:1026BD00BB010989828A83F8E028F022500327F7AD
:1026CD0022BBFE05F8E328F3228A838982F8E4937E
:0226DD002822B1
:1026DF00BB010689828A83F0225002F722BBFE01DA
:0226EF00F322D4
:1026F100F8BB010DE58229F582E5833AF583E8F01F
:10270100225006E92582C8F622BBFE05E92582C8CA
:02271100F222B2
:10271300EF8DF0A4A8F0CF8CF0A428CE8DF0A42EDA
:02272300FE2294
:10272500BC000BBE0029EF8DF084FFADF022E4CC98
:10273500F875F008EF2FFFEE33FEEC33FCEE9DEC61
:10274500984005FCEE9DFE0FD5F0E9E4CEFD22EDA7
:10275500F8F5F0EE8420D21CFEADF075F008EF2FF1
:10276500FFED33FD4007985006D5F0F222C398FDE2
:052775000FD5F0EA227F
:10277A00C2D5EC30E709B2D5E4C39DFDE49CFCEE7A
:10278A0030E715B2D5E4C39FFFE49EFE122725C3A6
:10279A00E49DFDE49CFC800312272530D507C3E4A1
:0627AA009FFFE49EFE22E9
:1027B000C5F0F8A3E028F0C5F0F8E58215827002B4
:0627C0001583E038F02251
:1027C600A3F8E0C5F025F0F0E582158270021583C6
:0627D600E0C838F0E82223
:1027DC00BB010A89828A83E0F5F0A3E022500687C8
:1027EC00F009E71922BBFE07E3F5F009E31922898A
:0B27FC00828A83E493F5F074019322BD
:10280700BB0110E58229F582E5833AF583E0F5F00F
:10281700A3E0225009E92582F886F008E622BBFEEC
:102827000AE92582F8E2F5F008E222E5832AF58332
:08283700E993F5F0A3E99322F7
:10283F00BB010A89828A83F0E5F0A3F0225006F7E4
:0F284F0009A7F01922BBFE06F3E5F009F31922E1
:10285E00EB9FF5F0EA9E42F0E99D42F0E89C45F0D0
:01286E002247
:10286F00E8600FEFC333FFEE33FEED33FDEC33FCC7
:03287F00D8F1226B
:102882007401FF3395E0FEFDFCA3A3A3E0CF2FF07C
:10289200E582158270021583E0CE3EF0E582158254
:1028A20070021583E0CD3DF0E5821582700215833A
:0528B200E0CC3CF02227
:0C28B700ECF0A3EDF0A3EEF0A3EFF02294
:1028C300A8828583F0D083D0821228DA1228DA1204
:1028D30028DA1228DAE473E493A3C583C5F0C58329
:1028E300C8C582C8F0A3C583C5F0C583C8C582C85F
:0128F30022C2
:1028F400F5F0C582A4C582C5F0C583A42583F583FC
:0129040022B0
:0C290500A42582F582E5F03583F58322DD
:10291100D083D082F8E4937012740193700DA3A355
:1029210093F8740193F5828883E473740293686069
:06293100EFA3A3A380DF69
:062937008A838982E4732B
:102A4200E51B248EF582E43404F583E0051B229015
:102A5200048B30170390048EE475F00112293D02B5
:102A620026772010E97F2ED2108018EF540F249081
:102A7200D43440D4FF30140BEF24BFB41A005003F7
:102A82002461FFE51C6002151C051FE51F7002058D
:102A92001E30170E90048BE475F00112293DEF02EF
:102AA20026DF025D4B7403D2178003E4C217F51BC5
:102AB20090048B122954E4F51CF51EF51FE51C60E9
:102AC200077F20122A8580F5751DFFC211C210C230
:102AD20012C213C215C216C218122A51FF700D304B
:102AE20017057F00122A96AF1FAE1E22B4255FC2C1
:102AF200D5C214122A51FF24D0B40A00501A75F01C
:102B02000A781C30D50508B6FF0106C6A426F620B1
:102B1200D5047002D21380D924CFB41A00EF500426
:102B2200C2E5D214022C97D21180C6D21080C0D234
:102B32001280BCD2D580BAD21580B47F20122A85E9
:102B42002012077401B51C0040F1122A42FF122A1A
:102B520085022ABFD218D2168095122A42FB122A67
:102B620042FA122A42F94A4B700679687A2D7BFFA3
:102B720020122EE51C602A7E008E827583001226AA
:102B82009060060EEE651D70F0C2D5EBC0E0EAC0A3
:102B9200E0E9C0E0EE122CDED0E0F9D0E0FAD0E0BD
:102BA200FB122677FF60AAEBC0E0EAC0E0E9C0E0D2
:102BB200122A85D0E02401F9D0E03400FAD0E0FBFB
:102BC200E51D0460DCD51DD980877BFF7A2C79DA7C
:102BD200D212809C791080027908C216C21880082D
:102BE200D2D5790A8004790AC2D5E51D047002F5AE
:102BF2001DE4FAFDFEFF122A42FC7B08201113128B
:102C02002A42FD7B1030100A122A42FE122A42FF8B
:102C12007B20EC3382D592D55013C3E43010069F4B
:102C2200FFE49EFEE42011039DFDE49CFCE4CBF84E
:102C3200C211EC700CCFCECDCCE824F8F870F38042
:102C420017C3EF33FFEE33FEED33FDEC33FCEB3312
:102C5200FB994002FB0FD8E9EB301105F8D0E0C434
:102C620048B211C0E00AEC4D4E4F78207B0070C292
:102C7200EAB51D0040BCC0E0122CE0D0F0D0E0204C
:102C82001104C4C0E0C4B211C0F0122A6ED0F0D553
:102C9200F0EB022ABF1229112B5C532BD6582B2D95
:102CA2004C2B29422BDA4F2BE2442BE2492B424395
:082CB2002BE8552BCC462BCC7E
:102CBA00452BCC472D88502B312D2B352E2B582BBD
:102CCA002B39232B56202D712A2AF14800002B502C
:102CDA003F3F3F00790AA2D5201314301509B910D5
:102CEA00020404B9080104A2D520160250010420E6
:102CFA0012689212B51C005034C0E07F20301319BC
:102D0A007F30A21272167215500F122D37C212C2DC
:102D1A0016C215C2187F30800F301503E9C0E012C1
:102D2A002A85301503D0E0F9D0E0B51CCC30151750
:102D3A007F30B9100C122A857F583014077F7880AB
:102D4A0003B90803122A853012057F2D022A857FCE
:102D5A00202018F87F2B2016F322921280CF286E9B
:102D6A00756C6C2900D211122A423011F8C21178FE
:102D7A001C30D50108F6022AF12D50434958122A6F
:102D8A00422403B405004001E4902D8393122A766D
:0D2D9A00743A122A76D213751C04022BD64F
:10293D00F8E0FBA3A3E0F925F0F0E5821582700223
:07294D001583E0FA38F022C7
:09295400EBF0A3EAF0A3E9F02284
:105D4B00EFB40A07740D125D56740A309811A899B6
:105D5B00B8130CC2983098FDA899C298B811F630B8
:075D6B0099FDC299F5992290
:00000001FF
